:020000040000FA
:04000000E7EF02F034
:04000800FFEF12F004
:0800180054EF13F00F0B756E9D
:10002000000EF76E360EF66E7550F626D8B0F72A2B
:100030000800F55012003031323334353637383954
:10004000414243444546000EF86E270EF76EB80E47
:10005000F66E96EC0DF0A5EC16F076EC00F003E3EE
:100060004C6A4D6A04D00AC24CF00BC24DF028EC29
:1000700019F09FEC1AF087EC1DF01FEC21F0040E34
:100080006B6E020E6C6EC1EC20F012EF20F0000ED1
:10009000F86E270EF76EA80EF66E96EC0DF07DC08A
:1000A000AAF17EC0ABF17FC0ACF180C0ADF181C0E0
:1000B000AEF179EC22F0EEEC22F076EC00F013E3F6
:1000C0004C6A4D6A4E6A4F6A506A4CC0AFF14DC0DF
:1000D000B0F14EC0B1F14FC0B2F150C0B3F1030E58
:1000E0004C6E4CC0B9F1BEEC24F0120081C04CF053
:1000F000D8804CAED890120089EC00F0D5EC01F01D
:100100009EEC01F077EC01F023EC00F047EC00F0FE
:100110001200000EF86E270EF76E860EF66E96EC45
:100120000DF0A5EC16F01CC04CF01DC04DF007EC16
:1001300021F0030E6B6E12EC20F0000EF86E270E0D
:10014000F76E8A0EF66E96EC0DF0A5EC16F01BC05D
:100150004CF007EC21F0030E6B6E12EC20F01A66E7
:1001600010D0000EF86E270EF76EC60EF66E96ECE7
:100170000DF0000EF86E270EF76ECC0EF66E96ECB4
:100180000DF0010E1A6210D0000EF86E270EF76EF9
:10019000D20EF66E96EC0DF0000EF86E270EF76E8E
:1001A000D80EF66E96EC0DF0020E1A6210D0000E0C
:1001B000F86E270EF76EDE0EF66E96EC0DF0000E62
:1001C000F86E270EF76EE40EF66E96EC0DF0030E49
:1001D0001A6210D0000EF86E270EF76EEA0EF66E59
:1001E00096EC0DF0000EF86E270EF76EF00EF66E20
:1001F00096EC0DF0040E1A6210D0000EF86E270E69
:10020000F76EF60EF66E96EC0DF0000EF86E270EF9
:10021000F76EFC0EF66E96EC0DF0050E1A6210D01D
:10022000000EF86E280EF76E020EF66E96EC0DF0CC
:10023000000EF86E280EF76E080EF66E96EC0DF0B6
:100240001200000EF86E270EF76E960EF66E96EC04
:100250000DF0A5C161F0A6C162F0A7C163F0A8C10D
:1002600064F0A9C165F01FEC21F0050E6B6E010E64
:100270006C6EC1EC20F012EC20F0040EF5EC0CF0EA
:10028000000EF86E270EF76EA20EF66E96EC0DF0CD
:100290009BC161F09CC162F09DC163F09EC164F09E
:1002A0009FC165F01FEC21F0050E6B6E010E6C6EA8
:1002B000C1EC20F012EC20F084EC0DF0A0C161F054
:1002C000A1C162F0A2C163F0A3C164F0A4C165F052
:1002D0001FEC21F0050E6B6E010E6C6E6E84C1EC8E
:1002E00020F012EC20F06A0EF5EC0CF01200540E27
:1002F00082EC0DF0460EF5EC0CF031503009F5ECC7
:100300000CF03A0EF5EC0CF0A5EC16F0C5C14CF073
:10031000C6C14DF00A0E516EA7EC1EF007EC21F09D
:10032000050E6B6E6F8612EC20F0000EF86E280E34
:10033000F76E120EF66E9AEC0DF01200356608D0CC
:10034000000EF86E270EF76E5E0EF66E96EC0DF050
:10035000010E356208D0000EF86E270EF76E660E9D
:10036000F66E96EC0DF0030E356208D0000EF86EB6
:10037000270EF76E6E0EF66E96EC0DF0040E3562DB
:1003800008D0000EF86E270EF76E760EF66E96EC1D
:100390000DF0020E356208D0000EF86E270EF76ED3
:1003A0007E0EF66E96EC0DF01200000EF86E270E23
:1003B000F76EB40EF66E96EC0DF0A5EC16F02FC0AD
:1003C0004CF007EC21F0010E6B6E12EF20F0716E15
:1003D000670E82EC0DF07150F5EF0CF0235202E144
:1003E000078C2FD081A0FAD7060E716E20EC0CF08E
:1003F00081A026D0712EFAD71EEC0CF04C6A080EA4
:10040000716E81A009D0D8804C32235202E1078C52
:1004100018D081B0FAD708D0D8904C32235202E1DC
:10042000078C0FD081A0FAD71CEC0CF0712EE9D705
:10043000235202E1078C05D081B0FAD7D89001D0C1
:10044000D8801200079C12EE0CF0130E726E736AC5
:1004500073C0E6FF722EFCD73E0EE7EC01F012EE01
:100460000CF0130E726E736A320E236EB7DF07BC88
:1004700047D04CC0E6FF722EF7D7120E716E12EE07
:100480000CF0516AE6CF4CF04C50511A712EFAD74D
:1004900051C073F0E7CFE8FF515C0AE0000EF86E40
:1004A000270EF76EBE0EF66E96EC0DF0078C28D078
:1004B00012EE0CF0E6CF4CF0AA0E4C5CFBE0E552DD
:1004C000E6CF2FF0E6CF1AF0E6CF1BF0E6CF1CF018
:1004D000E6CF1DF0E6CF0AF2E6CF0BF2E6CF7DF0D5
:1004E000E6CF7EF0E6CF7FF0E6CF80F0E6CF81F07A
:1004F000E6CFC5F1E6CFC6F1E6CF31F0E6CFC9F1E0
:10050000200EE7EC01F007821200350E0C6EA3EC12
:1005100009F014EC0CF0380E0C6EA3EC09F014EC9E
:100520000CF00C0E0C6EA3EC09F018EC0CF022ECA5
:1005300002F00880140E2A6E12001F0E82EC0DF0DD
:100540005B0EF5EC0CF010EE10F0060E716EE6CFBF
:100550004CF00A0E4C6203D02A0E4C6E14D00B0ED7
:100560004C6203D0300E4C6E0ED00C0E4C6203D099
:10057000230E4C6E08D0000E4C6203D0200E4C6E41
:1005800002D0300E4C124C50F5EC0CF0712EDFD72F
:100590005D0EF5EC0CF01200106A116A126A136A13
:1005A000146A156A10EE10F0E1CF0EF0E2CF0FF0F2
:1005B0001200D2EC02F00788320E226E520EE7ECE7
:1005C00001F0078A0880140E2A6E2D6812002EECA6
:1005D0000CF0ADEC0EF07CEC0CF06FEC0EF07CEC63
:1005E00000F0CCEC02F09DEC02F0520EE7EC01F0D2
:1005F0000C0E0C6EA3EC09F006EC0CF0050E2E6E42
:1006000085EC02F007AC2ED07AEC0DF0000EF86EFF
:10061000290EF76E7A0EF66E96EC0DF0000EF86E5F
:10062000290EF76E900EF66E96EC0DF0000EF86E39
:10063000290EF76EA60EF66E96EC0DF0000EF86E13
:10064000290EF76EBC0EF66E96EC0DF02E503009AA
:10065000F5EC0CF002EC0CF07AEC0DF07CEC00F018
:100660002E2ECED77CEC00F02E8CA1EC0DF0D8A075
:100670008CD3B4EC0DF00F0E0C6498D07AEC0DF026
:10068000190E0C6221D0000EF86E280EF76E280E9F
:10069000F66E96EC0DF0000EF86E280EF76E380E22
:1006A000F66E96EC0DF0000EF86E280EF76E4E0EFC
:1006B000F66E96EC0DF0000EF86E280EF76E640ED6
:1006C000F66E96EC0DF056D0180E0C6221D0000E8E
:1006D000F86E280EF76E7A0EF66E96EC0DF0000EA0
:1006E000F86E280EF76E8C0EF66E96EC0DF0000E7E
:1006F000F86E280EF76EA20EF66E96EC0DF0000E58
:10070000F86E280EF76EB80EF66E96EC0DF032D03D
:10071000170E0C6221D0000EF86E280EF76ECE0E6A
:10072000F66E96EC0DF0000EF86E280EF76EE00EE9
:10073000F66E96EC0DF0000EF86E280EF76EF60EC3
:10074000F66E96EC0DF0000EF86E290EF76E0C0E9C
:10075000F66E96EC0DF00ED0000EF86E280EF76EC9
:100760001E0EF66E96EC0DF00CC0E8FF0F0B300974
:10077000F5EC0CF00CC00DF019EC0EF008EC0CF0E0
:1007800014EC0EF0B4EC0DF00CC0E8FF0F0B3009C8
:10079000F5EC0CF00D38F00B0D6E0C500F0B0D122C
:1007A000BAEC0EF07AEC0DF00C6AEFD20EC0E1FF5D
:1007B0000FC0E2FF0CC0E6FFE1CF0EF0E2CF0FF07A
:1007C0001A0E0E5CD8B4D2EC02F00C0E0C6203D000
:1007D000D9EC02F002D09EEC09F0A3EC09F00C0E6B
:1007E000106203D0D9EC02F0226A050E106228D004
:1007F000090E116225D00C0E126222D0226A0798CF
:100800007AEC0DF0000EF86E290EF76EF60EF66E0D
:1008100096EC0DF0000EF86E2A0EF76E0C0EF66ECA
:1008200096EC0DF0000EF86E290EF76ECC0EF66EFB
:1008300096EC0DF014EC0EF07AEC0DF0CCEC02F02E
:10084000070E106205D0CCEC02F01B661B0638D0F8
:100850000A0E106206D0CCEC02F01B2A01E11B68E4
:100860002FD0080E106208D0CCEC02F01A2A060E27
:100870001A5C01E11A6A24D0060E10620ED0CCEC8C
:1008800002F01C6603D01D6601D006D01C061C2891
:10089000D8B41D06D8B41C5213D0090E106212D061
:1008A000CCEC02F0830E4C6E030E4D6E1D504D5C71
:1008B00002E11C504C5CD8B403D01C2AD8B41D2AC9
:1008C00089EC00F0040E106226D0090E116223D0CC
:1008D0000C0E126220D07AEC0DF0000EF86E2A0E8B
:1008E000F76E220EF66E96EC0DF0000EF86E2A0EE4
:1008F000F76E380EF66E96EC0DF0000EF86E2B0EBD
:10090000F76E980EF66E96EC0DF097EC09F07AEC17
:100910000DF0D9EC02F0040E10622AD0050E11621F
:1009200027D00C0E126201D003D00C0E136220D01F
:100930007AEC0DF0000EF86E2A0EF76E220EF66EAF
:1009400096EC0DF0000EF86E2A0EF76E4E0EF66E57
:1009500096EC0DF0000EF86E2B0EF76E980EF66EFC
:1009600096EC0DF097EC09F07AEC0DF0D9EC02F072
:10097000040E106289D0060E116286D07AEC0DF05A
:10098000000EF86E2A0EF76E220EF66E96EC0DF043
:10099000000EF86E2A0EF76E640EF66E96EC0DF0F1
:1009A0000C0E126209D0000EF86E2A0EF76E7A0E47
:1009B000F66E96EC0DF02BD00C0E136265D00B0E7C
:1009C000126211D0000EF86E2A0EF76E640EF66EEB
:1009D00096EC0DF0000EF86E2A0EF76EBE0EF66E57
:1009E00096EC0DF014D0000EF86E2A0EF76EA60EDF
:1009F000F66E96EC0DF012503009F5EC0CF0000E8E
:100A0000F86E2A0EF76EB60EF66E96EC0DF0000E2E
:100A1000F86E2A0EF76EEA0EF66E96EC0DF008EC04
:100A20000CF08A8285EC09F00BE2000EF86E2B0EBA
:100A3000F76E000EF66E96EC0DF08CEC09F002E30A
:100A400019EC0EF08A927AEC0DF0000EF86E2A0E78
:100A5000F76E220EF66E96EC0DF0000EF86E2A0E72
:100A6000F76E640EF66E96EC0DF0000EF86E2A0E20
:100A7000F76ED40EF66E96EC0DF006EC0CF07AECF8
:100A80000DF00884D9EC02F0040E10625CD0070E61
:100A9000116259D07AEC0DF0000EF86E2A0EF76E46
:100AA000220EF66E96EC0DF0000EF86E2A0EF76E22
:100AB000900EF66E96EC0DF00C0E126244D0000E05
:100AC000F86E2A0EF76E7A0EF66E96EC0DF0000EAA
:100AD000F86E2A0EF76EEA0EF66E96EC0DF008EC44
:100AE0000CF08A8285EC09F00BE2000EF86E2B0EFA
:100AF000F76E000EF66E96EC0DF08CEC09F002E34A
:100B000019EC0EF08A927AEC0DF0000EF86E2A0EB7
:100B1000F76E220EF66E96EC0DF0000EF86E2A0EB1
:100B2000F76E900EF66E96EC0DF0000EF86E2A0E33
:100B3000F76ED40EF66E96EC0DF006EC0CF07AEC37
:100B40000DF0D9EC02F0050E106232D0010E1162E8
:100B50002FD00C0E13622CD07AEC0DF0000EF86E34
:100B60002A0EF76E220EF66E96EC0DF0000EF86E61
:100B70002B0EF76E160EF66E96EC0DF0000EF86E5C
:100B80002B0EF76EAE0EF66E96EC0DF0000EF86EB4
:100B90002B0EF76EC40EF66E96EC0DF01250300967
:100BA000F5EC0CF097EC09F07AEC0DF0D9EC02F0D2
:100BB000050E106239D0020E116236D00C0E14628E
:100BC00033D07AEC0DF0000EF86E2A0EF76E220E7E
:100BD000F66E96EC0DF0000EF86E2B0EF76ECA0E48
:100BE000F66E96EC0DF0000EF86E2B0EF76EAE0E54
:100BF000F66E96EC0DF0140E82EC0DF012503009EA
:100C0000F5EC0CF0000EF86E2B0EF76EC40EF66EBF
:100C100096EC0DF013503009F5EC0CF097EC09F060
:100C20007AEC0DF0D9EC02F0050E106229D0040E1A
:100C3000116226D0070E126223D00C0E136220D050
:100C40007AEC0DF0000EF86E2A0EF76E220EF66E9C
:100C500096EC0DF0000EF86E2B0EF76E420EF66E4F
:100C600096EC0DF0000EF86E2B0EF76E980EF66EE9
:100C700096EC0DF097EC09F07AEC0DF0D9EC02F05F
:100C8000050E106229D0040E116226D0090E1262E0
:100C900023D00C0E136220D07AEC0DF0000EF86E0B
:100CA0002A0EF76E220EF66E96EC0DF0000EF86E20
:100CB0002B0EF76E2C0EF66E96EC0DF0000EF86E05
:100CC0002B0EF76E980EF66E96EC0DF097EC09F081
:100CD0007AEC0DF0D9EC02F0050E106226D0040E6D
:100CE000116223D00C0E126220D07AEC0DF0000EAF
:100CF000F86E2A0EF76E220EF66E96EC0DF0000ED0
:100D0000F86E2B0EF76E580EF66E96EC0DF0000E88
:100D1000F86E2B0EF76E980EF66E96EC0DF097ECC3
:100D200009F07AEC0DF0D9EC02F0050E106215D046
:100D3000040E116212D00B0E12620FD00C0E136251
:100D40000CD07AEC0DF0CCEC02F0079A226ABCECE5
:100D500008F07AEC0DF0D9EC02F0050E106212D01A
:100D6000050E11620FD00C0E12620CD07AEC0DF051
:100D7000CCEC02F0079A226A05EC09F07AEC0DF04F
:100D8000D9EC02F09DEC02F00C6A07BE06D080ECB4
:100D90000EF0D8A002D01AEC0AF02E4E2E8C010EC6
:100DA0002E6207D007A205D07CEC00F09DEC02F08B
:100DB0000792020E2E6214D007AE12D0AEEC0AF0EB
:100DC000079E346A010E35620BD0610E82EC0DF085
:100DD0002A0E07A6200EF5EC0CF00776C80E256E3D
:100DE000030E2E6208D0030E356205D0296603D0AB
:100DF000296864EC0EF0040E2E6207D008A005D01E
:100E00002A6603D008906BEC08F0050E2E6200D025
:100E1000060E2E6200D0070E2E6203D0256601D08A
:100E20000896080E2E620BD0010E356208D0266699
:100E300006D008A604D097EC0EF0640E266E090EBC
:100E40002E6211D0010E35620ED026660CD008B687
:100E50000AD0A2EC0EF012EC0CF097EC0EF0640E3F
:100E6000266EC80E256E0A0E2E6207D0246605D0A7
:100E700007A003D0BAEC09F007900B0E2E622FD01A
:100E800031A02DD007B02BD0C5C14CF0C6C14DF05C
:100E9000C7C151F0C8C152F0B80E536E0B0E546E5C
:100EA0005250545C02E15150535CD8A018D0AA0EA5
:100EB000536E000E546E5250545C02E15150535C1C
:100EC000D8B00DD052504D5C02E151504C5CD8B4BA
:100ED00006D0520EE7EC01F0640E246E07800C0E73
:100EE0002E620DD007AC0BD0079C320E236E23521E
:100EF00003E0A1EC0DF0FBE37AEC0DF007820D0EA0
:100F00002E6200D00E0E2E621BD0226619D007A8CA
:100F10000DD0106A116A126A136A146A156A166A89
:100F2000176A186A196A9DEC02F0079807AA08D098
:100F3000079A85EC02F008A403D0A2EC07F008940D
:100F400035EF03F0A5EC16F01CC04CF01DC04DF0C1
:100F5000640E516E1BEC1FF04CC074F0A5EC16F043
:100F60001CC04CF01DC04DF0716A746602D07182D5
:100F70004DD0010E746205D0640E516E7180718285
:100F800043D0020E746205D0C80E516E718071821A
:100F90003BD0030E746207D02C0E516E010E526EC0
:100FA0007180718231D0040E746207D0900E516E40
:100FB000010E526E7180718227D0050E746207D0C7
:100FC000F40E516E010E526E718071821DD0060EAC
:100FD000746207D0580E516E020E526E718071828B
:100FE00013D0070E746207D0BC0E516E020E526E03
:100FF0007180718209D0080E746206D0200E516E85
:10100000030E526E718000D023EC1AF071A006D04E
:101010000A0E4C6003D016EC08F007D071A205D080
:101020005A0E4C6402D037EC08F012007AEC0DF046
:1010300058EC08F0000EF86E2C0EF76E0C0EF66EE3
:1010400096EC0DF0000EF86E2C0EF76E2A0EF66E72
:1010500096EC0DF0000EF86E2C0EF76E560EF66E36
:1010600096EC0DF002EC0CF07AEC0DF012007AEC3C
:101070000DF058EC08F0000EF86E2C0EF76E0C0E0A
:10108000F66E96EC0DF0000EF86E2C0EF76E400E1C
:10109000F66E96EC0DF0000EF86E2C0EF76E560EF6
:1010A000F66E96EC0DF002EC0CF07AEC0DF01200FE
:1010B000000EF86E2C0EF76E220EF66E96EC0DF00A
:1010C000B3EC16F01CC04CF01DC04DF007EC21F045
:1010D000E6EC1FF0120019D83BC037F0790E366EDF
:1010E0009CEC08F03AC037F07A0E366E9CEC08F0B3
:1010F00039C037F07B0E366E9CEC08F038C037F004
:101100007C0E366E9CEC08F01200A5EC16F0C5C102
:101110004CF0C6C14DF0E80E516E030E526EA7ECB6
:101120001EF007EC21F042C038F043C039F044C053
:101130003AF045C03BF012007E0EA7EC08F036C036
:10114000E8FFA7EC08F037C0E8FFA7EF08F04C6E07
:101150008A940DD8080E716E4C32D8A08A94D8B0FB
:101160008A8405D8712EF8D78A8401D812009E0E81
:10117000096E092EFED71200000EF86E2A0EF76EC9
:10118000220EF66E96EC0DF0000EF86E2B0EF76E3A
:101190006E0EF66E96EC0DF0000EF86E2B0EF76EDE
:1011A000840EF66E96EC0DF0C9C14CF020EC19F0EF
:1011B0009FEC1AF01FEC21F0030E6B6E6C6A12ECC0
:1011C00020F0000EF86E2B0EF76E8E0EF66E96EC7B
:1011D0000DF0D30E4C6E20EC19F09FEC1AF01FECC2
:1011E00021F0030E6B6E6C6A12EC20F0C80E276EB5
:1011F000000E286E286603D0276601D005D0A1EC2A
:101200000DF0F8E3B4EC0DF0120089EC00F019ECED
:1012100012F0E4EC12F022EC09F047EC09F007ECD4
:1012200010F021EC01F0DC0E276E050E286E28660A
:1012300003D0276601D005D0A1EC0DF0F8E3B4ECA3
:101240000DF01200000EF86E270EF76E8E0EF66E81
:1012500096EC0DF005C261F006C262F007C263F0C1
:1012600008C264F009C265F01FEC21F0050E6B6E38
:10127000010E6C6EC1EC20F012EC20F0000EF86E46
:10128000280EF76E1A0EF66E9AEC0DF01200000E94
:10129000F86E270EF76E920EF66E96EC0DF000C209
:1012A00061F001C262F002C263F003C264F004C2E2
:1012B00065F01FEC21F0050E6B6E030E6C6EC1EC39
:1012C00020F012EC20F0000EF86E280EF76E160ECD
:1012D000F66E9AEC0DF01200000EF86E2B0EF76E03
:1012E000E00EF66E96EC0DF0000EF86E2B0EF76E1B
:1012F000F60EF66E96EC0DF0B4EC0DF0090E0C62E5
:1013000002D0D89001D0D8801200A1EC0DF003E2F9
:1013100081A0FBD7D890120081A002D0640E2C6E61
:10132000A1EC0DF003E22C66F7D7D890120012EC76
:101330000CF081B0FCD706EC0CF012000101C76B79
:10134000C86B000112000C38F00B306E8B8A8B8852
:10135000A00E306203D0B00E306E05D0B00E3062F9
:1013600002D0A00E306E30C08CFF8B9A12EC0CF0C5
:101370008B8A120005EC0AF03C0EE7EC01F09DECC4
:1013800002F0200E82EC0DF0A5EC16F0C7C14CF077
:10139000C8C14DF00A0E516EA7EC1EF007EC21F00B
:1013A00000EE44F011EE31F0030E406EEDCF3EF052
:1013B0003E383F6E7FEC20F03EC03FF07FEC20F0E7
:1013C000402EF4D711EE32F0050E716EE7CFE8FF34
:1013D000F5EC0CF0E6CF0CF0B6DF14EC0CF0712E4F
:1013E000F5D7230EF5EC0CF00C0E0C6EA3EC09F007
:1013F0007CEC00F0CCEC02F09DEC02F00CEC0CF07C
:1014000005EC0AF085EC02F012002A0EE7EC01F080
:1014100018EC0CF081A003D0500E2B6EF9D72B6680
:10142000FED7120023EE00F034C0D9FF32C0DFFF38
:10143000342A1200040E35620CD012EC0AF03B0E76
:10144000326202D0078E04D0FA0E346401D0078EC7
:101450001200020E35620CD012EC0AF0FD0E326260
:1014600002D0078E04D0FA0E346401D0078E120029
:10147000030E35620CD012EC0AF03B0E326202D041
:10148000078E04D0FA0E346401D0078E1200010ECC
:10149000356224D0346603D032C000F318D0010E78
:1014A000346203D032C001F312D0020E346203D092
:1014B00032C002F30CD0030E346203D032C003F307
:1014C00006D0040E346203D032C004F300D0342AB4
:1014D000050E346202D0078E08862FD0000E3562CA
:1014E0002CD07E0E325C02E1346A27D0346604D000
:1014F00032C033F0342A21D0790E335C05E11ED896
:101500001CE232C01EF019D07A0E335C05E116D809
:1015100014E232C01FF011D07B0E335C05E10ED80F
:101520000CE232C020F009D07C0E335C06E106D814
:1015300004E232C021F0078E00D0120032500F0BAF
:101540004C6E0A0E4C5C08E23250F00B4C6EA00E52
:101550004C5C02E2D8901200D8801200000E356276
:101560001FD01E52D8A4B9EF0AF01F52D8B4DBEF37
:101570000BF0B3EC16F020C04CF01FC04DF01EC0B5
:101580004EF005EC1AF0ADEC17F0BAEC16F00A0EBE
:10159000516E1BEC1FF042C0C7F143C0C8F10BD124
:1015A000010E356221D0A5EC16F003C34CF002C346
:1015B0004DF001C34EF000C34FF005EC1AF0ADEC56
:1015C00017F0BAEC16F00A0E516EA7EC1EF0BAEC4A
:1015D00016F0100E516E270E526E1BEC1FF042C01B
:1015E000C7F143C0C8F1E7D0030E356241D000C354
:1015F0004CF0460E4C62DFD001C34CF0410E4C6201
:1016000001D003D0420E4C6220D0A5EC16F008C3E6
:1016100042F007C343F006C344F005C345F0D4ECE1
:1016200021F005EC1AF001C34CF0410E4C6205D0DC
:1016300042C078F043C079F019D0420E4C6205D018
:1016400042C07AF043C07BF011D0540E4C620ED0F1
:1016500002C37CF0310E7C6205D07AC0C7F17BC03A
:10166000C8F104D078C0C7F179C0C8F12968A3D007
:10167000020E35623BD000C34CF0FE0E4C629BD094
:1016800001C34CF0FE0E4C6296D002C34CF0000E2B
:101690004C6291D003C34CF0940E4C628CD004C3C6
:1016A0004CF0000E4C6287D00AC34CF0FD0E4C6229
:1016B00082D0A5EC16F005C34CF006C34DF007C36D
:1016C0004EF008C34FF009C350F005EC1AF0ADEC32
:1016D00017F0BAEC16F0100E516E270E526E1BEC7E
:1016E0001FF042C0C7F143C0C8F165D0040E356297
:1016F00062D000C34CF0460E4C622ED001C34CF0B9
:10170000410E4C6201D003D0420E4C6251D00DC349
:101710004CF03B0E4C624CD0A5EC16F008C342F0E6
:1017200007C343F006C344F005C345F0D4EC21F0F1
:1017300005EC1AF001C34CF0410E4C6205D042C0DA
:1017400078F043C079F021D0420E4C627ED742C07F
:101750007AF043C07BF019D05A0E4C6229D001C3F5
:101760004CF05A0E4C6224D002C34CF0530E4C6223
:101770001FD003C34CF0570E4C621AD005C34CF077
:101780003B0E4C6215D004C37CF07C6602D0300E58
:101790007C6E310E7C6205D07AC0C7F17BC0C8F187
:1017A00007D0300E7C6204D078C0C7F179C0C8F190
:1017B000346ADBEF0BF00880140E2A6E1200140E50
:1017C00082EC0DF0B3EC16F078C04CF079C04DF01F
:1017D00007EC21F012EC20F0540E82EC0DF0B3EC8B
:1017E00016F07AC04CF07BC04DF007EC21F012EC03
:1017F00020F0400E82EC0DF07C50F5EC0CF008EC83
:101800000CF0120006EC0CF008EC0CF008EC0CF0FC
:101810000EEC0CF00EEC0CF00EEC0CF0FA0E12D0FC
:10182000C80E10D0640E0ED0320E0CD01E0E0AD090
:101830000A0E08D0050E06D0030E04D0020E02D008
:10184000010E00D00B6E060E0A6EF80E096E092E00
:10185000FED70A2EFCD70B2EF6D712000D0EC16E46
:10186000BE0EC06E1F0E926E010E936E800E946EB1
:10187000000E956E070E966E000ED06EC00EF26EC4
:10188000400EF16E000EF06E010E9D6E000EA06E09
:10189000220ED56E910ECD6E000ECA6E000EB16E88
:1018A0001F0E806E010E816EF00E826E000E836E32
:1018B000070E846E11D8000ECE6E4C0ECF6E05EE64
:1018C00000F015EE00F0EACF83F0E9CF82F0E2CF2E
:1018D00085F0E1CF84F01200716A00EE00F0EE6A4C
:1018E000712EFDD7040E726E01EE00F0EE6A712EBD
:1018F000FDD7722EFBD7120080A61200809A839229
:10190000839014EC0CF0200E55EC0DF0800E55EC8D
:101910000DF018EC0CF0200E55EC0DF0800E55EC8F
:101920000DF020EC0CF0060E47EC0DF00C0E47EC21
:101930000DF0140E47EC0DF015EC0DF0A2EC0CF0D0
:101940007AEF0DF07AEC0DF0000EF86E2C0EF76EBB
:101950006C0EF66E96EC0DF0000EF86E2C0EF76E17
:10196000820EF66E96EC0DF0000EF86E2C0EF76EF1
:10197000980EF66E96EC0DF0000E356208D0000E53
:10198000F86E2C0EF76EAE0EF66E96EC0DF0010EA4
:10199000356208D0000EF86E2C0EF76EC40EF66E8F
:1019A00096EC0DF0030E356208D0000EF86E2C0E8A
:1019B000F76ED00EF66E96EC0DF0040E356208D080
:1019C000000EF86E2C0EF76EE20EF66E96EC0DF031
:1019D000020E356208D0000EF86E2C0EF76EF40E73
:1019E000F66E96EC0DF006EF0CF03C6E65EC0DF02B
:1019F0003C5083828390809AF00B55EC0DF03C387C
:101A0000F00B53D03C6E3C463C463C4665EC0DF03A
:101A10003C50400947EC0DF0080E716E0900F5507E
:101A2000F5EC0CF0712EFAD7120080A61200000E11
:101A3000F86E1A0EF76E4E0EF66E080E726E736A20
:101A4000735002EC0DF0732A722EFAD712000000C8
:101A50000E11110A1B0000001010100001150000EB
:101A600014141400011500001515150001150E11B0
:101A700011110A0A1B000000000000000000000015
:101A8000000000000000000000000000000080A630
:101A900012003C6E65EC0DF03C50F00B839283908D
:101AA000809A55EC0DF03C38F00B80A61200E83817
:101AB0000F0B82B8100982BA200982BC400982BE8D
:101AC0008009826E808A809A120080A61200828627
:101AD0009486839283806E96808A000082A66E86AA
:101AE000809A0000808A0000809A6EA6F4D79496AF
:101AF00083901200010ECBD7020EC9D7800EC7D734
:101B0000C00EC5D78009C3D7200E6FD7716E84EC85
:101B10000DF0712EFCD712003D6E3D380EEC00F03A
:101B2000F5EC0CF03D500EEC00F05FD70900F550DD
:101B300082EC0DF00900F55003E0F5EC0CF0FAD75B
:101B40001200AAEC0DF00BEC0EF002E0D88001D0F0
:101B5000D89012008B808B828B848B8612008B90A6
:101B60008B928B948B961200A1EC0DF0FDE30C6A26
:101B7000E7EC0DF00C6E040E716E18EC0CF0E7EC57
:101B80000DF00C62F1D7712EF8D7000E0CB807D00B
:101B9000030E0CBA04D0060E0CBC01D0090E726EF6
:101BA000010E0CB404D0020E0CB201D0030E72264A
:101BB00072C00CF0500E716EA1EC0DF006E318EC43
:101BC0000CF0712EF9D7100E0C262D681200AFEC18
:101BD0000DF08B800BEC0EF015E1AFEC0DF08B826D
:101BE0000BEC0EF00FE1AFEC0DF08B840BEC0EF074
:101BF00009E1AFEC0DF08B860BEC0EF003E1726A9D
:101C0000E86A12008250E838F00B726E0BEC0EF0AE
:101C10007210AFEF0DF08450070BE8A002D0040E55
:101C200002D0E8B4010E12000C6AA1EC0DF0FCE346
:101C30001200A1EC0DF0FDE212001D0E0DD0190EE8
:101C40000BD0150E09D0110E07D00D0E05D0090EC0
:101C500003D0050E01D0010EC26EC282C2B2FED701
:101C6000C4CF77F0C3CF76F01200A6B2FED705C07E
:101C7000A9FF06C0A8FFA69EA69CA684F29EF2BE5F
:101C8000FDD7550EA76EAA0EA76EA68207A4F28EE8
:101C9000A6941200A6B2FED705C0A9FFA69EA69CD8
:101CA000A680A8CF06F01200DECF06F035EC0EF0CD
:101CB000052A712EF9D712004AEC0EF006C0DEFF9D
:101CC000052A712EF9D71200410E7CEC0EF0490E58
:101CD0007CEC0EF0320E7CEC0EF03B0E0DD0030EC1
:101CE000356202D03B0E01D01D0EAF6EAC94AC8AB3
:101CF000AB88AB8E9D8A12009EA8FED7AD6E1200F7
:101D000084C0E1FF85C0E2FF8251E15C02E1D8902E
:101D10001200E650326EF10EE15C02E115EE00F0C9
:101D2000E1CF84F0E2CF85F03250D8801200010E6E
:101D3000356207D0346A040E716E09D8030E7CEF49
:101D40000EF01200010E356207D0050E716EE86AC2
:101D50007CEC0EF0712EFBD71200056A4AEC0EF0F7
:101D600006C035F0120035C006F0056A35EC0EF0FD
:101D700012EF0CF0910E0D6203D0000E356E2CD0D8
:101D8000920E0D6203D0010E356E26D0930E0D62B9
:101D900003D0020E356E20D0940E0D6203D0030ED8
:101DA000356E1AD0950E0D6203D0040E356E14D028
:101DB0008B0E0D6202D0EFEF0EF0810E0D6202D09D
:101DC0002EEF0FF0710E0D6202D06DEF0FF0720E5C
:101DD0000D6202D098EF0FF0C6DF078212007C6A16
:101DE0007AEC0DF00C6A0D6AA1EC0DF00CE3B4EC8A
:101DF0000DF00C0E0C6201D0FF000B0E0C6203D034
:101E00007AEC0DF07C6A80EC0EF0ECE3280E7C623C
:101E100001D07C6A7C6605D05FEC13F0000E82EC8A
:101E20000DF00A0E7C6205D068EC13F0400E82ECD7
:101E30000DF0140E7C6205D071EC13F0140E82ECE0
:101E40000DF01E0E7C6205D07AEC13F0540E82EC7D
:101E50000DF032508CEC0DF07C2AC4D77C6A7AEC01
:101E60000DF00C6A0D6AA1EC0DF00CE3B4EC0DF072
:101E70000C0E0C6201D0FF000B0E0C6203D07AEC4A
:101E80000DF07C6A80EC0EF0ECE3500E7C6201D029
:101E90007C6A7C6605D05FEC13F0000E82EC0DF0DE
:101EA000140E7C6205D068EC13F0400E82EC0DF04D
:101EB000280E7C6205D071EC13F0140E82EC0DF04C
:101EC0003C0E7C6205D07AEC13F0540E82EC0DF0DF
:101ED0003250F5EC0CF07C2AC4D77C6A7AEC0DF019
:101EE000000EF86E290EF76E0C0EF66E96EC0DF0E5
:101EF0000C6A0D6AA1EC0DF01AE3B4EC0DF01C0EA7
:101F00000C6201D0FF000A0E0C6202D02A0E0DD026
:101F10000B0E0C6202D0300E08D00C0E0C6202D0F8
:101F2000230E03D00CC0E8FF3009F5EC0CF0E0D72D
:101F30007C6A7AEC0DF0000EF86E290EF76E0C0E2E
:101F4000F66E96EC0DF0000EF86E290EF76E380E58
:101F5000F66E96EC0DF00C6A0D6AA1EC0DF056E3EE
:101F6000B4EC0DF01C0E0C6201D0FF000C0E0C62E4
:101F70004DD07AEC0DF0000EF86E290EF76E220EA1
:101F8000F66E96EC0DF008EC0CF07AEC0DF085ECAA
:101F900002F07AEC0DF012EE0CF00A0E716EE6CF44
:101FA000E8FF8CEC0DF0712EFAD7090E716E400E21
:101FB00082EC0DF0E6CFE8FF8CEC0DF0712EFAD735
:101FC00007BC09D0000EF86E290EF76E4E0EF66EA5
:101FD00096EC0DF008D0000EF86E290EF76E640E28
:101FE000F66E96EC0DF006EC0CF0000EF86E290E75
:101FF000F76E0C0EF66E96EC0DF0000EF86E290ED4
:10200000F76E380EF66E96EC0DF000D0A4D7E4EC27
:1020100012F019EC12F0A5EC16F0C5C14CF0C6C1D7
:102020004DF04C5204E14D5202E118EF12F028EC51
:1020300019F09FEC1AF0E7EC1CF035EC1BF0D8EC33
:102040001CF0B5EC1AF0BAEC1CF0B5EC1AF061C05B
:102050002CF162C02DF163C02EF164C02FF165C078
:1020600030F100C261F001C262F002C263F003C24B
:1020700064F004C265F02CC166F02DC167F02EC17A
:1020800068F02FC169F030C16AF0B5EC1AF061C098
:1020900091F162C092F163C093F164C094F165C0A4
:1020A00095F105C261F006C262F007C263F008C292
:1020B00064F009C265F02CC166F02DC167F02EC135
:1020C00068F02FC169F030C16AF0B5EC1AF061C058
:1020D00022F162C023F163C024F164C025F165C020
:1020E00026F109EC1DF0DCEC16F022C166F023C1EC
:1020F00067F024C168F025C169F026C16AF035ECAB
:102100001BF0658E61C096F162C097F163C098F1D3
:1021100064C099F165C09AF1010E1A6231D0B2EC37
:102120001CF066C04BF167C04CF168C04DF169C04E
:102130004EF16AC04FF191C150F192C151F193C17A
:1021400052F194C153F195C154F1616A626A636AB4
:10215000646A656A61C055F162C056F163C057F1A7
:1021600064C058F165C059F196C15AF197C15BF14D
:1021700098C15CF199C15DF19AC15EF1B2EC28F0B1
:10218000020E1A6244D0616A626A636A646A656AAE
:1021900061C050F162C051F163C052F164C053F1AB
:1021A00065C054F161C055F162C056F163C057F18A
:1021B00064C058F165C059F1B2EC1CF066C04BF137
:1021C00067C04CF168C04DF169C04EF16AC04FF173
:1021D00096C15AF197C15BF198C15CF199C15DF16B
:1021E0009AC15EF1B2EC28F00101556B566B576B4A
:1021F000586B596B000191C15AF192C15BF193C1C7
:102200005CF194C15DF195C15EF11CEC26F0030E0A
:102210001A6231D0B2EC1CF066C04BF167C04CF1D1
:1022200068C04DF169C04EF16AC04FF196C150F1DE
:1022300097C151F198C152F199C153F19AC154F12A
:10224000616A626A636A646A656A61C055F162C004
:1022500056F163C057F164C058F165C059F191C19E
:102260005AF192C15BF193C15CF194C15DF195C1EA
:102270005EF1B2EC28F0040E1A6244D0616A626A20
:10228000636A646A656A61C050F162C051F163C0FB
:1022900052F164C053F165C054F161C055F162C0A0
:1022A00056F163C057F164C058F165C059F1B2EC02
:1022B0001CF066C04BF167C04CF168C04DF169C0BD
:1022C0004EF16AC04FF191C15AF192C15BF193C1D5
:1022D0005CF194C15DF195C15EF1B2EC28F00101B1
:1022E000556B566B576B586B596B000196C15AF181
:1022F00097C15BF198C15CF199C15DF19AC15EF142
:102300001CEC26F01A6616D0B2EC1CF066C04BF13D
:1023100067C04CF168C04DF169C04EF16AC04FF121
:1023200091C150F192C151F193C152F194C153F155
:1023300095C154F1050E1A6216D0B2EC1CF066C0BD
:102340004BF167C04CF168C04DF169C04EF16AC0F5
:102350004FF196C150F197C151F198C152F199C115
:1023600053F19AC154F10101547F00014BC19BF11B
:102370004CC19CF14DC19DF14EC19EF14FC19FF1E9
:1023800050C1A0F151C1A1F152C1A2F153C1A3F1B9
:1023900054C1A4F14BC161F04CC162F04DC163F076
:1023A0004EC164F04FC165F04BC166F04CC167F09F
:1023B0004DC168F04EC169F04FC16AF0B5EC1AF03A
:1023C00061C00EF162C00FF163C010F164C011F181
:1023D00065C012F150C161F051C162F052C163F0A9
:1023E00053C164F054C165F050C166F051C167F04B
:1023F00052C168F053C169F054C16AF0B5EC1AF0EB
:102400000EC166F00FC167F010C168F011C169F02C
:1024100012C16AF078EC1BF0E1EC1BF061C0A5F191
:1024200062C0A6F163C0A7F164C0A8F165C0A9F1BC
:102430001200A5EC16F01CC04CF01DC04DF028ECAD
:1024400019F09FEC1AF0F2EC16F01CC04CF01DC015
:102450004DF0640E516E000E526E52504D5C02E112
:1024600051504C5CD8B001D08DD0C80E516E000ECA
:10247000526E52504D5C02E151504C5CD8B001D0CC
:1024800054D02C0E516E010E526E52504D5C02E132
:1024900051504C5CD8B001D048D0900E516E010E16
:1024A000526E52504D5C02E151504C5CD8B001D09C
:1024B0003CD0F40E516E010E526E52504D5C02E152
:1024C00051504C5CD8B001D030D0580E516E020E35
:1024D000526E52504D5C02E151504C5CD8B001D06C
:1024E00024D0BC0E516E020E526E52504D5C02E171
:1024F00051504C5CD8B001D018D0200E516E030E54
:10250000526E52504D5C02E151504C5CD8B001D03B
:102510000CD0840E516E030E526E52504D5C02E18F
:1025200051504C5CD8B001D000D0B3EC16F051C083
:102530004CF052C04DF028EC19F09FEC1AF0E7EC8B
:102540001CF072EC1BF076EC17F0E7EC1CF072EC70
:102550001BF081EC17F0D1EC16F008EC17F072ECE0
:102560001BF03F0E6A6EB30E696E330E686E330E4B
:10257000676E330E666EB5EC1AF01EEC17F078EC51
:102580001BF00ED0D1EC16F03E0E6A6EBD0E696ED9
:10259000700E686EA30E676ED70E666EB5EC1AF0FD
:1025A000410E6A6E880E696E666A676A686A78ECC0
:1025B0001BF061C005F262C006F263C007F264C09E
:1025C00008F265C009F21200A5EC16F01BC04CF031
:1025D00028EC19F09FEC1AF03E0E6A6E666A676A84
:1025E000686A696AB5EC1AF061C000F262C001F273
:1025F00063C002F264C003F265C004F21200EACFC5
:1026000004F0E9CF03F083C0EAFF82C0E9FF9EAA8D
:102610000ED0AE50ABA204D0AE50AB98AB88F7D77B
:10262000EE6EF10EE95C02E105EE00F0F0D7EACFC4
:1026300083F0E9CF82F0F2A402D0F29430D0F2A27B
:1026400002D0F2922CD09EA022D09E90226622062A
:1026500023662306246624062566250626662606A6
:10266000286602D0275206E027062728D8B4280675
:10267000D8B42752296629062A662A062B662B0615
:102680002C662C06000ECE6E4C0ECF6E08D0A1A884
:1026900002D0A19804D09EA202D09E9200D004C085
:1026A000EAFF03C0E9FF1100006ED8CF01F0E0CFD0
:1026B00002F002C0E0FF005001C0D8FF1000000E81
:1026C000F86E270EF76E060EF66E96EC0DF0120001
:1026D000000EF86E270EF76E1C0EF66E96EC0DF0DF
:1026E0001200000EF86E270EF76E320EF66E96ECA4
:1026F0000DF01200000EF86E270EF76E480EF66E03
:1027000096EC0DF012000020202020202020202018
:1027100020202020202020202020200040202020B9
:1027200020202020202020202020202020202020A9
:1027300020001420202020202020202020202020C5
:102740002020202020202000542020202020202075
:1027500020202020202020202020202020000B507E
:102760005374617200000B465438343700000B4B31
:102770003220202000000B507753445200000A49B9
:1027800043373330300000433A00404C3A000A43AC
:102790003A004A4C3A0014496D706564616E7A3DA6
:1027A0002000545A3D20000014503A0054463A008C
:1027B00054663A0011413A004B5357523A002043B5
:1027C000524320213D00062D4C2D000046202020A4
:1027D0000000062D4C2B0000462020430000062B55
:1027E0004C2D0000464320200000062D432B000006
:1027F0004620204C0000062B432D0000464C202094
:102800000000062D432D00004620202000004D48EA
:102810007A006B487A00754800007046000000425C
:10282000656665686C3A2000005452582052656D08
:102830006F74653A20390000405B315D5069636117
:1028400053746172205B345D4B3220202000145B96
:10285000325D4654383437202020205B355D507778
:1028600053445200545B335D4943373330302020AA
:10287000202020202020202000000052533233321C
:10288000204D6F6E69746F723A203800405B305D86
:102890002048657864657A696D616C20202020206D
:1028A0002000145B315D2041736363692020202088
:1028B0002020202020202000545B235D20416262E4
:1028C00072756368202020202020202020000054E2
:1028D000657366756E6B74696F6E656E3A2037004E
:1028E000405B315D2054617374656E66656C642075
:1028F000202020202000145B325D204C45442D44D4
:102900006174656E7472616E73662E00545B232071
:102910006C616E675D20416262727563682121207F
:10292000200000446174656E6162727566202D2D11
:102930002D3E202020202000145B235D2044617464
:10294000656E616272756620202020202000143D93
:102950003D3D3D206572666F6C67726569636820F6
:102960003D3D3D00143D3D3D3D206665686C657212
:1029700068616674203D3D3D3D00003D204B65692A
:102980006E6520446174656E20766F6D203D200079
:10299000403D20416E74656E6E656E2D54756E659A
:1029A0007221203D2000143D2057617274656E2015
:1029B000352053656B212020203D2000543D2056BA
:1029C0006572737563683A203D200000543D20779E
:1029D0006569746572206D69742022232220203D70
:1029E00020001F435243206F6B2100001F435243BE
:1029F00020213D200000003D3D3D3D2053796D5498
:102A0000756E6572203D3D3D3D3D2000403D3D20C1
:102A1000696D20536C6565706D6F647573203D3D05
:102A20003D00003D3D3D3D3D2046756E6B74696F38
:102A30006E203D3D3D3D3D00402D2D20537065698C
:102A4000636865726E2042616E64202D2D00402DFA
:102A5000537065692E31306B487A205365676D6518
:102A60006E742D00402D2D2D2D204E6163687475E0
:102A70006E656E202D2D2D2D2D00142D2062697375
:102A800020535752204D696E696D756D202D2D00B4
:102A9000402D2054756E656E20696E20466C616510
:102AA000636865202D00142D2D2D2062697320533D
:102AB000575220312C0023202D2D2D2D0000142DB8
:102AC0002D20696E20466C61656368652038783812
:102AD000202D2D00542D2D2D2D2054756E656E202A
:102AE000617573202D2D2D2D2D00542D2D20576116
:102AF0007274656E205458204F4E202D2D2D2D00C0
:102B0000542D2D2057617274656E205458204F4605
:102B100046202D2D2D00402D2D416E74656E6E6565
:102B2000206C6F65736368656E2D2D00402D2050FD
:102B300049436565202D2D3E206578746565202DFF
:102B40002D00402D206578746565202D2D3E205088
:102B500049436565202D2D00402D20506F7765720B
:102B60002C2053575220434C52202D2D2D00402D08
:102B70002D2D2046572056657273696F6E656E2045
:102B80002D2D2D001454756E6572203A000054529C
:102B9000656D6F74653A0000142057617274656E3C
:102BA00020626973204C45442061757321005420D4
:102BB00057617274656E20626973204C45442061D0
:102BC00075732100162D2D3E2000402D2D416E7471
:102BD000656E6E65206B6F70696572656E2D2D0078
:102BE00014205B395D204F4B205765697465722056
:102BF00020202020200054205B235D20416262724F
:102C00007563682020202020202020000042656677
:102C10002E343620776965646572686F6C656E2145
:102C200020004043776572743D0014696E2074691A
:102C300065666572656E204265726569636820002D
:102C400014696E20686F65686572656E20426572F2
:102C5000656963682000546D6974204265662E348E
:102C600033207765636873656C6E21000053796D5E
:102C700054756E65722044544D462D52656D6F74C7
:102C80006500404857312E303220202032302E311E
:102C9000312E323032312000145357322E31312D43
:102CA00034353230202020444C344A414C005443C7
:102CB00041542D506963415374617220444C344A2D
:102CC000414C2000544341542D46542038343700A1
:102CD000544341542D4B3220456C656372616674D8
:102CE0000000544341542D50432D506F776572536B
:102CF00044520000544341542D494337333030206F
:102D000049636F6D00002D2D2D00494E46006D5713
:102D10000000755700006E5700007057000066579E
:102D2000000061570000572000006B57000020563C
:102D300000006D560000755600006E56000064429B
:102D40006D00644200007373000013D806D8476A10
:102D5000486A496A4A6A4B6A1200426A436A446A8C
:102D6000456A466A12004C6A4D6A4E6A4F6A506A5A
:102D70001200F9DF516A526A536A546A556A1200A6
:102D8000616A626A636A646A656A12000EC166F00B
:102D90000FC167F010C168F011C169F012C16AF08B
:102DA00012000EC161F00FC162F010C163F011C1D9
:102DB00064F012C165F0120066C061F067C062F095
:102DC00068C063F069C064F06AC065F0120061C059
:102DD00066F062C067F063C068F064C069F065C007
:102DE0006AF0120061C00EF162C00FF163C010F111
:102DF00064C011F165C012F1120013C161F014C179
:102E000062F015C163F016C164F017C165F01200DD
:102E100013C166F014C167F015C168F016C169F0FE
:102E200017C16AF0120018C161F019C162F01AC12D
:102E300063F01BC164F01CC165F0120018C166F09C
:102E400019C167F01AC168F01BC169F01CC16AF0B2
:102E500012001DC161F01EC162F01FC163F020C1EC
:102E600064F021C165F012001DC166F01EC167F05B
:102E70001FC168F020C169F021C16AF0120022C1AF
:102E800061F023C162F024C163F025C164F026C162
:102E900065F0120022C166F023C167F024C168F01A
:102EA00025C169F026C16AF0120027C161F028C16E
:102EB00062F029C163F02AC164F02BC165F01200F1
:102EC00027C166F028C167F029C168F02AC169F0FE
:102ED0002BC16AF0120066C013F167C014F168C01C
:102EE00015F169C016F16AC017F1120061C013F143
:102EF00062C014F163C015F164C016F165C017F12A
:102F0000120061C018F162C019F163C01AF164C007
:102F10001BF165C01CF1120061C01DF162C01EF101
:102F200063C01FF164C020F165C021F1120061C0CF
:102F300022F162C023F163C024F164C025F165C0B1
:102F400026F1120061C027F162C028F163C029F1A7
:102F500064C02AF165C02BF1120042C04CF043C09E
:102F60004DF044C04EF045C04FF046C050F0120046
:102F700042C051F043C052F044C053F045C054F039
:102F800046C055F012004CC042F04DC043F04EC058
:102F900044F04FC045F050C046F012005136523652
:102FA00053365436553612004C364D364E364F3663
:102FB00050361200553254325332523251321200CE
:102FC00050324F324E324D324C32120006D8473614
:102FD000483649364A364B36120042364336443676
:102FE0004536463612004B324A3249324832473271
:102FF0001200F9DF46324532443243324232120087
:103000004CAE04D04D684E684F68506812004DAE0B
:1030100003D04E684F68506812004EAE02D04F6821
:10302000506812004FAE01D0506812006F926EBE11
:103030006F828CDE280E3F6ED890E0EC17F0FAEC31
:1030400017F003D83F2EF8D71200E9EC21F00A0E52
:103050003E6E00EE42F0EF50E8B6FD0FE8BED00F36
:10306000EE6E3E2EF8D7F6EC21F012003FD846AEB9
:1030700009D0472AD8B4482AD8B4492AD8B44A2A09
:10308000D8B44B2AADEC16F035D030D846AE09D0C6
:10309000472AD8B4482AD8B4492AD8B44A2AD8B436
:1030A0004B2A47C042F048C043F049C044F04AC0F0
:1030B00045F04BC046F06EBEEEEC1EF0120016D886
:1030C00047C042F048C043F049C044F04AC045F010
:1030D0004BC046F06EBEEEEC1EF0120007D8A7EC17
:1030E00016F008D003D8ADEC16F004D089EC1AF035
:1030F0007EEF18F03BEC19F09FEF1AF04CD803E18B
:10310000A6EC16F01AD01AD87F0E566E56505A5E9C
:1031100057505B5A5AC03EF05A520FE05ABE06D082
:10312000D890E6EC17F03E2EFBD707D03E1E3E2A85
:10313000D890F9EC17F03E2EFBD712006E9E60BEC1
:103140006E8E609EA6EC16F05CC043F05DC044F04D
:103150005EC045F05FC046F060C047F0D890E6EC36
:1031600017F0FAEC17F0468E47C05AF0476AD8902D
:10317000E6EC17F01200040E3E6EEE6608D03E2E0E
:10318000FCD7EECFE8FF7F0B03E1D88401D0D894C1
:10319000F6EC21F01200E9EC21F000EE5CF0EBD748
:1031A000E9EC21F000EE61F0E6D7E9EC21F000EE69
:1031B00066F0E1D7E9EC21F000EE4CF0DCD7E9EC69
:1031C00021F000EE51F0D7D7E9EC21F000EE42F00B
:1031D0000A0E3E6EEE66DBD73E2EFCD7D6D7506A7F
:1031E0004FBE506835D04F6A506A4EAE31D04F68EE
:1031F00050682ED04E6A4F6A506A4DAE29D04E6844
:103200004F68506825D04D6A4E6A4F6A506A4CAE7E
:103210001FD04D684E684F6850681AD0A6EC16F063
:103220006E9E506A1DD0A6EC16F06E9E4F6A506AD4
:1032300017D0A6EC16F06E9E4E6A4F6A506A10D0F8
:10324000A6EC16F06E9E4D6A4E6A4F6A506A08D020
:10325000A6EC16F06E9E50AE03D0FDEC1EF06E8E06
:103260004CC047F04DC048F04EC049F04FC04AF046
:1032700050C04BF000D07F0E5A6E000E5B6EE4EC37
:1032800018F006E15C6A5D6A5E6A5F6A606A36D061
:10329000A5EC19F007E0D890F9EC17F05A2AD8B449
:1032A0005B2AF6D747B00AD0D890E6EC17F05A065A
:1032B0005A28D8B45B06D8B45A52F4D743A00BD0DE
:1032C0004380432AD8B4442AD8B4452AD8B4462ADD
:1032D000D8B4472ADDD7426A47905AC047F0F9EC84
:1032E00017F043C05CF044C05DF045C05EF046C0DE
:1032F0005FF047C060F0609E6EBE608E12005C6A38
:103300005D6A5E6A606A800E5F6EF5D75C685D68B4
:103310005E687F0E5F6E7F0E606EEDD77F0E4C6E27
:10332000000E4D6E5B504D5C02E15A504C5CD8B0C3
:1033300003D0ECDFD88401D0D89412005BAE03D068
:10334000DEDFD88401D0D8941200E9EC21F000EE41
:103350004BF0040E3E6EED660AD03E2EFCD7010EF9
:10336000EF6201D002D0EF6602D0D88401D0D894A9
:10337000F6EC21F0120051C000F152C001F153C02F
:1033800002F154C003F155C004F105EC1AF042C03B
:1033900007F143C008F144C009F145C00AF146C035
:1033A0000BF100C14CF001C14DF002C14EF003C160
:1033B0004FF004C150F0EBEC19F007C147F008C121
:1033C00048F009C149F00AC14AF00BC14BF06E9EAA
:1033D0006FB26E8E1200BADC280E3F6ED89005D800
:1033E000EDEC17F03F2EFAD71200E9EC21F0050EB4
:1033F0003E6E00EE4CF0D890EF50E8200700EE6EE5
:103400003E2EFAD7F6EC21F01200E9EC21F09EDC1A
:10341000280E3F6ED890E0EC17F0FAEC17F000EEB3
:103420004CF0050E3E6EEFAE02D0300EEF5EEFA612
:1034300002D0030EEF5EEE523E2EF5D73F2EEAD7B6
:10344000F6EC21F0120002D8ADEF17F0E9EC21F014
:103450009ADD00EE42F010EE51F0040E3E6EE650A2
:10346000EE5EE650EE5A3E2EFCD7F6EC21F012004E
:1034700002D8ADEF17F0E9EC21F085DD00EE42F067
:1034800010EE51F0E650EE26040E3E6EE650EE22AF
:103490003E2EFCD7F6EC21F0120000C14CF001C129
:1034A0004DF002C14EF003C14FF004C150F005C110
:1034B00056F006C157F0120007C151F008C152F092
:1034C00009C153F00AC154F00BC155F00CC158F0BA
:1034D0000DC159F0120043C000F144C001F145C0D4
:1034E00002F146C003F147C004F15AC005F15BC0C8
:1034F00006F1120043C007F144C008F145C009F1CC
:1035000046C00AF147C00BF15AC00CF15BC00DF187
:10351000120061C05CF062C05DF063C05EF064C028
:103520005FF065C060F0120066C05CF067C05DF0DF
:1035300068C05EF069C05FF06AC060F012005CC0F5
:1035400061F05DC062F05EC063F05FC064F060C0B7
:1035500065F012005CC066F05DC067F05EC068F0A8
:103560005FC069F060C06AF0120006EC22F016E25B
:1035700003EC22F013E2D0EC18F01AE0D5EC18F0CE
:1035800017E01BEC22F004E3D0EC18F001E306D0C6
:103590001EEC22F006E3D5EC18F003E343EC22F036
:1035A00012001BEC22F003E338EC22F003D00DD024
:1035B000C0EC16F065BE03D06AAE01D0658E65AE74
:1035C00003D06ABE01D0658E12001DD86E9E6EBA01
:1035D0006E7E6EBC6E7EAAEC1EF046C000F147C047
:1035E00001F148C002F149C003F14AC004F11ED8FC
:1035F0003BEC1AF0ADEC17F0BAEC16F07F0E516E02
:1036000026EC1AF01ED06E9A6E9C65BE6E8A6ABE5B
:103610006E8C7FDF9EEC18F05EDF86DF9EEC18F08C
:1036200069DFA5EC16F039DF5CEF1AF0A5EC16F0B7
:1036300056C04CF057C04DF058C051F059C052F030
:10364000120042C05AF043C05BF0A6EC16F000C175
:1036500043F001C144F002C145F003C146F004C18A
:1036600047F03FEC19F09FEF1AF006EC22F009E268
:1036700003EC22F006E2D0EC18F006E1D5EC18F0ED
:1036800019E143EC22F012001EEC22F003E31BECE4
:1036900022F0F7E2D5EC18F010E138EC22F065BE2C
:1036A00003D06AAE01D0658E65AE03D06ABE01D08C
:1036B000658E12004DEC22F0F2D7A5DF6E9E6EBA39
:1036C0006E7E6EBC6E7E78EC1FF005DFAFDF26EC01
:1036D0001AF0ADEC17F0BAEC16F07F0E516E3BEC21
:1036E0001AF0AFD7D5EC18F001E112006A7E00D0D5
:1036F00006EC22F004E203EC22F001E203D043ECFA
:1037000022F01200D5EC18F001E11200D0EC18F014
:1037100003E1DCEC16F0120017D83BEC1AF056C0AF
:103720005AF057C05BF06E9E46AE03D06E8EEEEC44
:103730001EF042C000F143C001F144C002F145C097
:1037400003F146C004F181D75EDFFE0E5A6E000E13
:103750005B6E5950575C02E15850565C27E013E30A
:10376000582AD8B4592A5B50595C02E15A50585C27
:1037700007E1BAEC16F056C058F057C059F016D011
:10378000D89018DCE6D7562AD8B4572A5B50575C35
:1037900002E15A50565C07E1B3EC16F058C056F0FF
:1037A00059C057F003D0D8900BDCD3D76EBAFDECDC
:1037B0001EF06EBC0CEC1FF01200E7EC16F0B5EF3B
:1037C0001AF0D0EC18F02DE065BE2CD006EC22F0FB
:1037D00028E2F2EC16F0ECD848DF76EC17F01E0E7B
:1037E000416E414E1ED0D1EC16F008EC17F03DDFD3
:1037F00008EC17F07DDFDCD838DF08EC17F06A50F2
:10380000655C0BE16950645C08E16850635C05E14C
:103810006750625C02E16650615C03E076EC17F091
:10382000E0D7120043EC22F01200D0EC18F008E1CF
:103830003F0E656E800E646E616A626A636A120092
:1038400001013F0E266F800E256F226B236B246BC8
:103850003F0E216F800E206F1D6B1E6B1F6B0001D2
:1038600081EC17F076EC17F022C10EF123C10FF1B5
:1038700024C110F125C111F126C112F11E0E416EB5
:10388000FDEC16F034EC17F0F0DEC6EC16F078EC38
:103890001BF0C6EC16F06A50655C0BE16950645C85
:1038A00008E16850635C05E16750625C02E16650C4
:1038B000615C17E0414E15D0F2EC16F03FEC17F0CA
:1038C0006FD816DF97EC17F034EC17F04EDE8CEC67
:1038D00017F013EC17F008EC17F047DE76EC17F052
:1038E000CFD71200D0EC18F008E13F0E656E800EC5
:1038F000646E616A626A636A120061C02CF162C020
:103900002DF163C02EF164C02FF165C030F16EEC73
:1039100018F03BD82ADE89DFA2EC17F02CC161F049
:103920002DC162F02EC163F02FC164F030C165F08B
:1039300076EC18F06E946EBE6E8447C041F027C1DD
:1039400061F028C162F029C163F02AC164F02BC183
:1039500065F0415206E06EA4C5D86EB4D5D8412EAC
:10396000FAD71200420E6A6E480E696E666A676A7E
:10397000686A1200400E6A6E490E696E0F0E686E1C
:10398000DA0E676EA20E666E1200400E6A6E130E9D
:10399000696E5D0E686E8D0E676EDE0E666E1200CD
:1039A0003F0E6A6E800E696E666A676A686A120008
:1039B000400E6A6E666A676A686A696A1200410E3A
:1039C0006A6E200E696E666A676A686A1200420E45
:1039D0006A6EC80E696E666A676A686A1200440E8B
:1039E0006A6E7A0E696E666A676A686A1200460EC7
:1039F0006A6E1C0E696E400E686E666A676A120017
:103A0000470E6A6EC30E696E500E686E666A676A0C
:103A10001200490E6A6E740E696E240E686E666A34
:103A2000676A12004B0E6A6E180E696E960E686E0B
:103A3000800E676E666A12004C0E6A6EBE0E696E6C
:103A4000BC0E686E200E676E666A12004E0E6A6EBD
:103A50006E0E696E6B0E686E280E676E666A1200D7
:103A60003D0E6A6ECC0E696ECC0E686ECC0E676E23
:103A7000CD0E666E12003C0E6A6E230E696ED70E76
:103A8000686E0A0E676E3D0E666E12003A0E6A6E22
:103A9000830E696E120E686E6E0E676E980E666EFD
:103AA0001200350E6A6E860E696E370E686EBD0E98
:103AB000676E060E666E1200300E6A6E890E696EB3
:103AC000700E686E5F0E676E410E666E12002B0EF2
:103AD0006A6E8C0E696EBC0E686ECC0E676E090E37
:103AE000666E12006CDFB5EF1AF071DFB5EF1AF0F9
:103AF00076DFB5EF1AF07BDFB5EF1AF081DFB5EFB7
:103B00001AF087DFB5EF1AF05ADF35EF1BF05FDFF1
:103B100035EF1BF064DF35EF1BF069DF35EF1BF08D
:103B20006FDF35EF1BF075DF35EF1BF0D0EC18F0D1
:103B300003E143EC22F01200F2EC16F001013F0E1B
:103B4000176F800E166F136B146B156B000128DF57
:103B500072EC1BF081EC17F0D1EC16F021DF78EC61
:103B60001BF08CEC17F013EC17F034EC17F035EC7D
:103B70001BF081EC17F097EC17F0F2EC16F0280E22
:103B8000416EFDEC16F014DF78EC1BF076EC17F0CC
:103B900013EC17F04AEC17F0B5EC1AF04AEC17F0FA
:103BA000B5EC1AF081EC17F008EC17F035EC1BF0CF
:103BB000C6EC16F078EC1BF0C6EC16F06A50655CAB
:103BC0000BE16950645C08E16850635C05E1675093
:103BD000625C02E16650615C05E0414E03D0F2ECAC
:103BE00016F0CFD7E5DEB5EF1AF00101276B000123
:103BF000DFEC1CF048D806E384EC1DF00101272B14
:103C00000001F6D793DFC1DE35EC1BF0A5EC16F012
:103C100027C147F0475206E03BEC19F0AAEC1AF036
:103C200078EC1BF012007ED850AE14D055AE29D0DF
:103C30005AD85050555C0BE14F50545C08E14E503F
:103C4000535C05E14D50525C02E14C50515CD8B0E0
:103C500016D017D050BE02D055BE11D044D8505007
:103C6000555C0BE14F50545C08E14E50535C05E14C
:103C70004D50525C02E14C50515CD8B002D0D8900B
:103C800001D0D88012004ED850AE14D055AE29D0F5
:103C90002AD85050555C0BE14F50545C08E14E500F
:103CA000535C05E14D50525C02E14C50515CD8B080
:103CB00016D017D050BE02D055BE11D014D85050D7
:103CC000555C0BE14F50545C08E14E50535C05E1EC
:103CD0004D50525C02E14C50515CD8B002D0D880BB
:103CE00001D0D8901200D0EC18F003E1B3EC16F03C
:103CF0000FD0D890D4EC17F0D8904F324E324D32CE
:103D00004C324F8ED5EC18F003E1BAEC16F009D026
:103D1000D890CEEC17F0D890543253325232513200
:103D2000548E120061C04CF062C04DF063C04EF082
:103D300064C04FF065C050F066C051F067C052F0EB
:103D400068C053F069C054F06AC055F0120002D840
:103D5000ADEF17F0E9EC21F037D8050E3E6E00EE1E
:103D600051F020EE42F0A6EC16F010EE4CF0050EED
:103D70003F6E3EC040F03F50402640064006EF50A8
:103D8000E602F350DE26D9CF6BF0DACF6CF0F450B8
:103D9000DE22E86ADE22402EFCD76BC0D9FF6CC061
:103DA000DAFF3F2EE6D7EE5220EE42F0060E406ECE
:103DB0003E50405EDE52402EFDD73E2ED6D7F6EC6A
:103DC00021F06EB20BD812006E9250AE02D015D810
:103DD0006E7255AE02D020D86E721200421E431E83
:103DE000441E451E461E422AD8B4432AD8B4442A4B
:103DF000D8B4452AD8B4462A12004C1E4D1E4E1E79
:103E00004F1E501E4C2AD8B44D2AD8B44E2AD8B4CE
:103E10004F2AD8B4502A1200511E521E531E541E4F
:103E2000551E512AD8B4522AD8B4532AD8B4542A89
:103E3000D8B4552A1200C8DFE9EC21F0A6EC16F040
:103E4000050E3E6E00EE51F0EE6605D03E2EFCD71C
:103E5000F6EC21F012003E6A3E2AD89055BE1CD0E6
:103E6000513652365336543655365550505C0BE168
:103E700054504F5C08E153504E5C05E152504D5C8C
:103E800002E151504C5CE8E2A6EC16F0D8905532B5
:103E900054325332523251325550505C0BE154502F
:103EA0004F5C08E153504E5C05E152504D5C02E11D
:103EB00051504C5C0AE351504C5E52504D5A535095
:103EC0004E5A54504F5A5550505AEDEC17F03E2E62
:103ED000DDD777DF4CC051F04DC052F04EC053F0EB
:103EE0004FC054F050C055F0ADEC17F0F6EF21F094
:103EF000290E3E6EA6EC16F05550505C0BE1545066
:103F00004F5C08E153504E5C05E152504D5C02E1BC
:103F100051504C5C0BE351504C5E52504D5A535033
:103F20004E5A54504F5A5550505AD880E6EC17F01C
:103F3000D890D4EC17F05550505C0BE154504F5CC6
:103F400008E153504E5C05E152504D5C02E1515086
:103F50004C5C0BE351504C5E52504D5A53504E5AEC
:103F600054504F5A5550505AD8803E2EDFD7120029
:103F7000E9EC21F06E9250AE02D03FDF6E82A6ECEB
:103F800016F0280E3E6E0A0E3F6E00EE42F0EF5025
:103F90000F0B406E050E405CD8A002D0030EEF263A
:103FA000EF50F00B406E500E405CD8A002D0300EA7
:103FB000EF26EC523F2EEBD7D890D4EC17F0E6EC7E
:103FC00017F03E2EE0D7F6EC21F0120006EC22F0BE
:103FD00015E21EEC22F01CE22FD844D85AD86F9478
:103FE0001200030E6B6409D06C666B2A6EB46B2AE8
:103FF000030E6B5E6B5086EC0DF01200F2DF000ECC
:10400000F86E2D0EF76E060EF66E9AEC0DF012009D
:10401000E8DF000EF86E2D0EF76E0A0EF66E9AECC3
:104020000DF0120006EC22F0E9E21EEC22F0F0E2C4
:1040300003D82FD86F941200E9EC21F000EE4BF07A
:1040400011EE31F00A0E406EEDCF3EF03E383F6E7D
:1040500056D83EC03FF053D8402EF6D7E76AF6EC6C
:1040600021F01200E9EC21F06C5210E001EE44F076
:1040700011EE44F0140E3E6E6CC03FF0E5503E066B
:104080003F2EFCD7E5CFEDFF3E2EFCD7F6EC21F01E
:104090001200E9EC21F00A0E3F6E6C503F266B5087
:1040A0003F5CD8B002D03FC06BF06B506C5CD8A0C6
:1040B00003D06CC06BF06B2A6C506B5E6B06090E04
:1040C0003E6E6B503E5E01EE31F03E5204E0EECFAC
:1040D000E8FF3E2EFCD76EA405D02B0E6EBE2D0E33
:1040E000BEEC20F06E8019D86E9013D86C5204E0AC
:1040F0002C0EBEEC20F009D8F6EC21F012003F5057
:104100000F0B3009E8CFE6FF12006CC040F06F964D
:1041100006D0010E406E6F9602D06BC040F0405248
:1041200026E06EA006D0EFCF3EF0300E3E5CD8A465
:104130006E906FA611D040C04CF0020E4C6202D0BF
:10414000B8EC20F0050E4C6202D0B8EC20F0080E5E
:104150004C6202D0B8EC20F0EECFE8FF6EB003D096
:10416000BEEC20F002D0BAEC20F0402EDAD71200DC
:10417000200E04D0200E6FB4300E00D0F5EC0CF001
:104180001200E9EC21F00A0E3E6E6C503E5E00EE2D
:1041900042F0EF503E4E0CD0EF503E4E02D0EE5269
:1041A000F8D7EE524C6E490E4C6409D0010E06D081
:1041B0000F0B4C6E040E4C6402D0100EEF260A0E4C
:1041C0003E6E00EE42F0EF500700EE6EE86AEF221E
:1041D0003E2EF9D7F6EC21F01200E9EC21F0050EA5
:1041E0003E6E0A0E3F6E00EE4BF0EDCF4CF04C50A1
:1041F000F00B07E13F064C500F0B03E13F063E2E4C
:10420000F4D73FC04CF03F50F6EC21F012004DECDB
:1042100022F0A6EC16F0B8EC1FF042C047F043C005
:1042200048F044C049F045C04AF046C04BF0050E86
:104230006B6E6C6A6E946F946E986F96120006ECBB
:1042400022F044E21EEC22F041E289EC1AF07EEC0E
:1042500018F042C000F143C001F144C002F145C072
:1042600003F146C004F147C04CF048C04DF049C0CE
:104270004EF04AC04FF04BC050F0B8EC1FF042C0B7
:1042800007F143C008F144C009F145C00AF146C036
:104290000BF100C14CF001C14DF002C14EF003C161
:1042A0004FF004C150F016EC18F007C147F008C1F8
:1042B00048F009C149F00AC14AF00BC14BF0140E95
:1042C0006B6E0A0E6C6E6E986F966F946E94120001
:1042D000F2EC16F06D6A659ED0EC18F014E0DFEC9D
:1042E0001CF043EC1EF001E004E384EC1DF06D2AA9
:1042F000F6D7D0EC1CF013EC1EF005E004E372ECF2
:104300001DF06D06F6D71FEC21F0D1EC16F065BE5E
:104310006E8E0B0E6B6E0A0E6C6E6E846E981200B3
:1043200012EC20F0650EBEEC20F06E9E6DBE6E8E1F
:104330006DBE6D6CB3EC16F06DC04CF007EC21F067
:104340006E844BDF4CC06BF012EC20F01200FDECE1
:1043500016F0C6EC16F072EC1BF0A2EC17F029EC8C
:1043600017F01EEC17F072EC1BF0E7EC16F027C10B
:1043700061F028C162F029C163F02AC164F02BC149
:1043800065F035EC1BF0A2EC17F03FEC17F01EECDB
:1043900017F072EC1BF060EC17F0B5EC1AF0C6ECFD
:1043A00016F078EC1BF01200E9EC21F0B3EC16F0FB
:1043B000050E3E6E10EE42F020EE4CF0E6500F0B74
:1043C000DF6EE638F00BDE123E2EF8D7F6EC21F069
:1043D0001200E9CF45F1EACF46F1E1CF47F1E2CF54
:1043E00048F1D9CF49F1DACF4AF1120045C1E9FFCE
:1043F00046C1EAFF47C1E1FF48C1E2FF49C1D9FF19
:104400004AC1DAFF120094EC1AF003D089EC1AF0DA
:1044100000D0609E7F0E60620CD0800E5F6207D07D
:104420005E6605D05D6603D05C6601D002D0D880A0
:1044300001D0D890120094EC1AF003D089EC1AF055
:1044400000D0609E7F0E60620BD0800E5F6208D04D
:104450005E6606D05D6604D05C6602D0D88001D06E
:10446000D890120002D89FEF1AF005D8608E120083
:1044700002D89FEF1AF07F0E606E800E5F6E5C6A4E
:104480005D6A5E6A120002D89FEF1AF07F0E606EBE
:104490005C685D685E685F68120002D89FEF1AF082
:1044A0005C6A5D6A5E6A5F6A606A1200410E6A6EEB
:1044B000A00E696E666A676A686A120056EC22F09E
:1044C00035EC1BF072EC1CF0F2EC16F0D0EC1CF0AA
:1044D00078EC1BF076EC17F0D1EC16F0D0EC1CF079
:1044E00072EC1BF0E7EC16F0FDEC16F035EC1BF06F
:1044F0001200AAC161F0ABC162F0ACC163F0ADC102
:1045000064F0AEC165F084EC1DF072EC1CF061C08B
:10451000B4F162C0B5F163C0B6F164C0B7F165C073
:10452000B8F11200B4C161F0B5C162F0B6C163F078
:10453000B7C164F0B8C165F08AEC1DF0B2EC1CF0B4
:10454000B5EC1AF0E1EC1BF061C0BFF162C0C0F144
:1045500063C0C1F164C0C2F165C0C3F11200BFC144
:1045600061F0C0C162F0C1C163F0C2C164F0C3C1F7
:1045700065F00101010EC46F000151EC1DF013EC58
:104580001EF009E30101040EC46F000181EC1DF06F
:1045900078EC1DF018D046EC1DF013EC1EF007E38C
:1045A0000101030EC46F000181EC1DF00CD0D0ECB2
:1045B0001CF013EC1EF007E30101020EC46F0001B2
:1045C00078EC1DF000D061C0BAF162C0BBF163C0ED
:1045D000BCF164C0BDF165C0BEF11200B4C161F0B0
:1045E000B5C162F0B6C163F0B7C164F0B8C165F09F
:1045F0000101030EB96F000167EC1DF013EC1EF012
:104600000BE381EC1DF081EC1DF078EC1DF0010155
:10461000080EB96F00014CD05CEC1DF013EC1EF0DD
:1046200009E381EC1DF081EC1DF00101070EB96F6B
:1046300000013ED051EC1DF013EC1EF009E381ECBB
:104640001DF078EC1DF00101060EB96F000130D0AD
:1046500046EC1DF013EC1EF007E381EC1DF00101A8
:10466000050EB96F000124D0D0EC1CF013EC1EF045
:1046700007E378EC1DF00101040EB96F000118D0BA
:1046800009EC1DF043EC1EF007E393EC1DF0010173
:10469000010EB96F00010CD0EFEC1CF043EC1EF0E2
:1046A00007E38AEC1DF00101020EB96F000100D092
:1046B00061C0AFF162C0B0F163C0B1F164C0B2F1EA
:1046C00065C0B3F11200AFC161F0B0C162F0B1C119
:1046D00063F0B2C164F0B3C165F01FEC21F0050EC8
:1046E0006B6E010E6C6EDFEC1CF013EC1EF003E33E
:1046F000040E6C6E0FD0E7EC1CF013EC1EF003E31D
:10470000030E6C6E07D0EFEC1CF013EC1EF002E30E
:10471000020E6C6E67D8C1EC20F012EC20F0B9C12B
:104720004CF0030E4C6209D0000EF86E2D0EF76EA1
:104730000E0EF66E9AEC0DF054D0040E4C6209D0B9
:10474000000EF86E2D0EF76E120EF66E9AEC0DF04E
:1047500048D0050E4C6209D0000EF86E2D0EF76E93
:10476000160EF66E9AEC0DF03CD0060E4C6209D097
:10477000000EF86E2D0EF76E1A0EF66E9AEC0DF016
:1047800030D0070E4C6209D0000EF86E2D0EF76E79
:104790001E0EF66E9AEC0DF024D0020E4C6209D07B
:1047A000000EF86E2D0EF76E260EF66E9AEC0DF0DA
:1047B00018D0010E4C6209D0000EF86E2D0EF76E67
:1047C0002A0EF66E9AEC0DF00CD0080E4C6209D051
:1047D000000EF86E2D0EF76E220EF66E9AEC0DF0AE
:1047E00000D01200EDEC20F0030E4C6402D0010E5C
:1047F0006C6E030E4C6202D0020E6C6E020E4C62A6
:1048000002D0030E6C6E010E4C6202D0040E6C6E70
:10481000000E4C6202D0040E6C6E1200BAC161F040
:10482000BBC162F0BCC163F0BDC164F0BEC165F044
:104830001FEC21F0060E6B6E010E6C6EEFEC1CF09F
:1048400013EC1EF002E3020E6C6EE7EC1CF013ECAE
:104850001EF002E3030E6C6EDFEC1CF013EC1EF096
:1048600002E3040E6C6EBEDFC1EC20F012EC20F00F
:10487000C4C14CF0010E4C6209D0000EF86E2D0E32
:10488000F76E2E0EF66E9AEC0DF024D0020E4C62EE
:1048900009D0000EF86E2D0EF76E320EF66E9AEC01
:1048A0000DF018D0030E4C6209D0000EF86E2D0EDC
:1048B000F76E360EF66E9AEC0DF00CD0040E4C62CC
:1048C00009D0000EF86E2D0EF76E3A0EF66E9AECC9
:1048D0000DF000D01200AAC161F0ABC162F0ACC112
:1048E00063F0ADC164F0AEC165F01FEC21F0050EC0
:1048F0006B6E020E6C6EC1EC20F0EDEC20F0030E3E
:104900004C6004D0040E6B6E020E6C6E020E4C6492
:1049100004D0040E6B6E010E6C6E24D0AAC161F03F
:10492000ABC162F0ACC163F0ADC164F0AEC165F083
:104930001FEC21F0040E6B6E010E6C6EC1EC20F0CA
:10494000EDEC20F0030E4C6004D0030E6B6E010EF4
:104950006C6E020E4C6406D0040E6B6E000E6C6E14
:10496000C1EC20F06E8412EC20F0000EF86E2D0EDB
:10497000F76E3E0EF66E9AEC0DF01200AFC161F0CC
:10498000B0C162F0B1C163F0B2C164F0B3C165F00F
:104990001FEC21F0040E6B6E010E6C6EDFEC1CF050
:1049A00013EC1EF003E3030E6C6E0FD0E7EC1CF06B
:1049B00013EC1EF003E3020E6C6E07D0EFEC1CF05C
:1049C00013EC1EF002E3010E6C6EC1EC20F065D812
:1049D00012EC20F0B9C14CF0030E4C6209D0000E6D
:1049E000F86E2D0EF76E0E0EF66E9AEC0DF054D09A
:1049F000040E4C6209D0000EF86E2D0EF76E120EEA
:104A0000F66E9AEC0DF048D0050E4C6209D0000EFF
:104A1000F86E2D0EF76E160EF66E9AEC0DF03CD079
:104A2000060E4C6209D0000EF86E2D0EF76E1A0EAF
:104A3000F66E9AEC0DF030D0070E4C6209D0000EE5
:104A4000F86E2D0EF76E1E0EF66E9AEC0DF024D059
:104A5000020E4C6209D0000EF86E2D0EF76E260E77
:104A6000F66E9AEC0DF018D0010E4C6209D0000ED3
:104A7000F86E2D0EF76E2A0EF66E9AEC0DF00CD035
:104A8000080E4C6209D0000EF86E2D0EF76E220E45
:104A9000F66E9AEC0DF000D01200EDEC20F0030E53
:104AA0004C6404D0050E6B6E000E6C6E030E4C62EF
:104AB00002D0010E6C6E020E4C6202D0020E6C6EC1
:104AC000010E4C6202D0030E6C6E000E4C6202D0DE
:104AD000030E6C6E1200AFC161F0B0C162F0B1C1E3
:104AE00063F0B2C164F0B3C165F01FEC21F0030EB6
:104AF0006B6E010E6C6EDFEC1CF013EC1EF003E32A
:104B0000020E6C6E11D0E7EC1CF013EC1EF003E308
:104B1000010E6C6E09D0EFEC1CF013EC1EF004E3F8
:104B2000000E6C6E040E6B6EC1EC20F065D812ECBA
:104B300020F0B9C14CF0030E4C6209D0000EF86EA3
:104B40002D0EF76E0E0EF66E9AEC0DF054D0040E8C
:104B50004C6209D0000EF86E2D0EF76E120EF66E36
:104B60009AEC0DF048D0050E4C6209D0000EF86E9C
:104B70002D0EF76E160EF66E9AEC0DF03CD0060E6A
:104B80004C6209D0000EF86E2D0EF76E1A0EF66EFE
:104B90009AEC0DF030D0070E4C6209D0000EF86E82
:104BA0002D0EF76E1E0EF66E9AEC0DF024D0020E4E
:104BB0004C6209D0000EF86E2D0EF76E260EF66EC2
:104BC0009AEC0DF018D0010E4C6209D0000EF86E70
:104BD0002D0EF76E2A0EF66E9AEC0DF00CD0080E24
:104BE0004C6209D0000EF86E2D0EF76E220EF66E96
:104BF0009AEC0DF000D01200EDEC20F0030E4C64A6
:104C000004D0040E6B6E000E6C6E030E4C6204D06A
:104C1000040E6B6E000E6C6E020E4C6202D0010E22
:104C20006C6E010E4C6202D0020E6C6E000E4C6275
:104C300002D0020E6C6E12004BC161F04CC162F0EA
:104C40004DC163F04EC164F04FC165F055C166F0CF
:104C500056C167F057C168F058C169F059C16AF090
:104C600078EC1BF061C04BF162C04CF163C04DF1B8
:104C700064C04EF165C04FF150C161F051C162F0A6
:104C800052C163F053C164F054C165F05AC166F07B
:104C90005BC167F05CC168F05DC169F05EC16AF03C
:104CA00078EC1BF061C050F162C051F163C052F169
:104CB00064C053F165C054F112004BC161F04CC1A6
:104CC00062F04DC163F04EC164F04FC165F055C153
:104CD00066F056C167F057C168F058C169F059C114
:104CE0006AF072EC1BF061C04BF162C04CF163C022
:104CF0004DF164C04EF165C04FF150C161F051C13A
:104D000062F052C163F053C164F054C165F05AC1FE
:104D100066F05BC167F05CC168F05DC169F05EC1BF
:104D20006AF072EC1BF061C050F162C051F163C0D7
:104D300052F164C053F165C054F112004BC161F0EF
:104D40004CC162F04DC163F04EC164F04FC165F0DB
:104D500055C166F056C167F057C168F058C169F097
:104D600059C16AF0B5EC1AF061C00EF162C00FF1E2
:104D700063C010F164C011F165C012F150C161F05F
:104D800051C162F052C163F053C164F054C165F087
:104D90005AC166F05BC167F05CC168F05DC169F043
:104DA0005EC16AF0B5EC1AF061C013F162C014F193
:104DB00063C015F164C016F165C017F14BC161F015
:104DC0004CC162F04DC163F04EC164F04FC165F05B
:104DD0005AC166F05BC167F05CC168F05DC169F003
:104DE0005EC16AF0B5EC1AF061C018F162C019F149
:104DF00063C01AF164C01BF165C01CF150C161F0C1
:104E000051C162F052C163F053C164F054C165F006
:104E100055C166F056C167F057C168F058C169F0D6
:104E200059C16AF0B5EC1AF018C166F019C167F003
:104E30001AC168F01BC169F01CC16AF078EC1BF064
:104E400061C050F162C051F163C052F164C053F1CE
:104E500065C054F10EC161F00FC162F010C163F082
:104E600011C164F012C165F013C166F014C167F09E
:104E700015C168F016C169F017C16AF072EC1BF039
:104E800061C04BF162C04CF163C04DF164C04EF1A2
:104E900065C04FF112004BC161F04CC162F04DC1D1
:104EA00063F04EC164F04FC165F055C166F056C164
:104EB00067F057C168F058C169F059C16AF0B5ECA4
:104EC0001AF061C00EF162C00FF163C010F164C04E
:104ED00011F165C012F150C161F051C162F052C1CF
:104EE00063F053C164F054C165F05AC166F05BC110
:104EF00067F05CC168F05DC169F05EC16AF0B5EC55
:104F00001AF00EC166F00FC167F010C168F011C150
:104F100069F012C16AF078EC1BF061C00EF162C05A
:104F20000FF163C010F164C011F165C012F155C1F9
:104F300061F056C162F057C163F058C164F059C1C5
:104F400065F055C166F056C167F057C168F058C1A9
:104F500069F059C16AF0B5EC1AF061C013F162C092
:104F600014F163C015F164C016F165C017F15AC1A0
:104F700061F05BC162F05CC163F05DC164F05EC171
:104F800065F05AC166F05BC167F05CC168F05DC155
:104F900069F05EC16AF0B5EC1AF013C166F014C195
:104FA00067F015C168F016C169F017C16AF078ECB6
:104FB0001BF061C013F162C014F163C015F164C04D
:104FC00016F165C017F1E7EC16F00EC161F00FC1E4
:104FD00062F010C163F011C164F012C165F035ECEC
:104FE0001BF061C00EF162C00FF163C010F164C02C
:104FF00011F165C012F14BC161F04CC162F04DC1BD
:1050000063F04EC164F04FC165F05AC166F05BC1F8
:1050100067F05CC168F05DC169F05EC16AF0B5EC33
:105020001AF061C018F162C019F163C01AF164C0CE
:105030001BF165C01CF150C161F051C162F052C159
:1050400063F053C164F054C165F055C166F056C1B8
:1050500067F057C168F058C169F059C16AF0B5EC02
:105060001AF018C166F019C167F01AC168F01BC1C7
:1050700069F01CC16AF072EC1BF013C166F014C138
:1050800067F015C168F016C169F017C16AF035EC18
:105090001BF061C050F162C051F163C052F164C0B5
:1050A00053F165C054F10EC14BF10FC14CF110C169
:1050B0004DF111C14EF112C14FF112004BC15FF120
:1050C0004CC160F14DC161F14EC162F14FC163F15C
:1050D00050C164F151C165F152C166F153C167F12C
:1050E00054C168F112005FC14BF160C14CF161C164
:1050F0004DF162C14EF163C14FF164C150F165C120
:1051000051F166C152F167C153F168C154F1120007
:1051100055C169F156C16AF157C16BF158C16CF1C3
:1051200059C16DF15AC16EF15BC16FF15CC170F193
:105130005DC171F15EC172F1120069C155F16AC1C0
:1051400056F16BC157F16CC158F16DC159F16EC187
:105150005AF16FC15BF170C15CF171C15DF172C157
:105160005EF112005EEC28F088EC28F01CEC26F0D2
:105170004BC173F14CC174F14DC175F14EC176F163
:105180004FC177F150C178F151C179F152C17AF133
:1051900053C17BF154C17CF173EC28F09DEC28F0F5
:1051A0009EEC26F073C155F174C156F175C157F1EB
:1051B00076C158F177C159F178C15AF179C15BF1E3
:1051C0007AC15CF17BC15DF17CC15EF14BEC27F0F3
:1051D00012007AEC0DF060EC29F002EC0CF01200F9
:1051E0007AEC0DF04BC161F04CC162F04DC163F03F
:1051F0004EC164F04FC165F065508CEC0DF0645009
:105200008CEC0DF063508CEC0DF062508CEC0DF0DA
:1052100061508CEC0DF084EC0DF050C161F051C187
:1052200062F052C163F053C164F054C165F065503F
:105230008CEC0DF064508CEC0DF063508CEC0DF0A8
:1052400062508CEC0DF061508CEC0DF0400E82EC55
:105250000DF055C161F056C162F057C163F058C1FD
:1052600064F059C165F065508CEC0DF064508CEC25
:105270000DF063508CEC0DF062508CEC0DF0615031
:105280008CEC0DF084EC0DF05AC161F05BC162F062
:105290005CC163F05DC164F05EC165F065508CEC8B
:1052A0000DF064508CEC0DF063508CEC0DF06250FE
:1052B0008CEC0DF061508CEC0DF002EC0CF0120057
:1052C000000E4BC161F04CC162F04DC163F04EC1A4
:1052D00064F04FC165F00FD8400E50C161F051C16C
:1052E00062F052C163F053C164F054C165F003D859
:1052F0006A0EF5EF0CF082EC0DF01FEC21F00D0EB4
:105300006B6E070E6C6E6E84C1EC20F012EF20F015
:10531000400E4BC161F04CC162F04DC163F04EC113
:1053200064F04FC165F0E7DF140E50C161F051C168
:1053300062F052C163F053C164F054C165F0DBDF29
:105340006A0EF5EF0CF0140E4BC161F04CC162F027
:105350004DC163F04EC164F04FC165F0CCDF540E17
:1053600050C161F051C162F052C163F053C164F0A9
:0C53700054C165F0C0DF6A0EF5EF0CF0D0
:020000040030CA
:0300010002191EC3
:020005008184F4
:0200000400F00A
:020000000401F9
:00000001FF
